:0200000480007A
:100000006F000005732F2034930F80006308FF03F7
:10001000930F90006304FF03930FB0006300FF038E
:10002000130F000063040F0067000F00732F2034CC
:1000300063540F006F00400093E19153171F0000BD
:1000400023223FFC171F000023200FFC6FF01FFF2F
:100050009300000013010000930100001302000050
:100060009302000013030000930300001304000038
:100070009304000013050000930500001306000020
:100080009306000013070000930700001308000008
:10009000930800001309000093090000130A0000F0
:1000A000930A0000130B0000930B0000130C0000D8
:1000B000930C0000130D0000930D0000130E0000C0
:1000C000930E0000130F0000930F0000732540F102
:1000D0006310050097020000938202017390523072
:1000E000735044749702000093820201739052305F
:1000F00073500018970200009382420273905230AE
:100100009B021000939252039382F2FF7390023B82
:100110009302F0017390023A73504030970200004E
:1001200093824201739052307350203073503030BC
:100130009301000097020000938202ED7390523009
:10014000130510001315F501635C05000F00F00F97
:10015000930110009308D005130500007300000000
:1001600093020000638A020073905210B7B200003D
:100170009B829210739022307350003097020000DF
:100180009382420173901234732540F17300203042
:100190009301200093000000130100003B87200022
:1001A000930300006316774C930130009300100016
:1001B000130110003B87200093032000631A774A45
:1001C0009301400093003000130170003B87200032
:1001D0009303A000631E7748930150009300000032
:1001E0003781FFFF3B872000B783FFFF631277480B
:1001F00093016000B7000080130100003B872000DE
:10020000B70300806316774693017000B700008043
:100210003781FFFF3B872000B783FF7F631A774456
:100220009301800093000000378100001B01F1FF63
:100230003B872000B78300009B83F3FF631A77425C
:1002400093019000B70000809B80F0FF1301000035
:100250003B872000B70300809B83F3FF631A77403E
:100260009301A000B70000809B80F0FF3781000061
:100270001B01F1FF3B872000B78300809B83E3FFD6
:100280006318773E9301B000B7000080378100000B
:100290001B01F1FF3B872000B78300809B83F3FFA6
:1002A0006318773C9301C000B70000809B80F0FF8B
:1002B0003781FFFF3B872000B783FF7F9B83F3FFDE
:1002C0006318773A9301D000930000001301F0FF08
:1002D0003B8720009303F0FF631C77389301E00015
:1002E0009300F0FF130110003B87200093030000F0
:1002F000631077389301F0009300F0FF1301F0FFD3
:100300003B8720009303E0FF6314773693010001DD
:1003100093001000370100801B01F1FF3B87200094
:10032000B703008063167734930110019300D00067
:100330001301B000BB80200093038001639A7032E8
:10034000930120019300E0001301B0003B812000E5
:1003500093039001631E7130930130019300D0002C
:10036000BB8010009303A00163947030930140019F
:10037000130200009300D0001301B0003B8720005F
:10038000130307001302120093022000E31452FE2D
:1003900093038001631E732C93015001130200002C
:1003A0009300E0001301B0003B8720001300000021
:1003B000130307001302120093022000E31252FEFF
:1003C000930390016316732A9301600113020000E6
:1003D0009300F0001301B0003B87200013000000E1
:1003E0001300000013030700130212009302200001
:1003F000E31052FE9303A001631C73269301700166
:10040000130200009300D0001301B0003B872000CE
:100410001302120093022000E31652FE93038001A0
:100420006318772493018001130200009300E00019
:100430001301B000130000003B87200013021200DC
:1004400093022000E31452FE93039001631277227B
:1004500093019001130200009300F0001301B0001B
:1004600013000000130000003B872000130212005D
:1004700093022000E31252FE9303A001631A771E39
:100480009301A001130200009300D00013000000AC
:100490001301B0003B8720001302120093022000DA
:1004A000E31452FE930380016314771C9301B0019F
:1004B000130200009300E000130000001301B000DD
:1004C000130000003B87200013021200930220005B
:1004D000E31252FE93039001631C77189301C0014D
:1004E000130200009300F00013000000130000004E
:1004F0001301B0003B87200013021200930220007A
:10050000E31252FE9303A001631477169301D00106
:10051000130200001301B0009300D0003B872000BD
:100520001302120093022000E31652FE930380018F
:10053000631077149301E001130200001301B0006F
:100540009300E000130000003B872000130212001C
:1005500093022000E31452FE93039001631A771074
:100560009301F001130200001301B0009300F000AA
:1005700013000000130000003B872000130212004C
:1005800093022000E31252FE9303A0016312770E40
:1005900093010002130200001301B00013000000D9
:1005A0009300D0003B87200013021200930220002A
:1005B000E31452FE93038001631C770A9301100237
:1005C000130200001301B000130000009300E000CC
:1005D000130000003B87200013021200930220004A
:1005E000E31252FE930390016314770893012002F3
:1005F000130200001301B0001300000013000000FC
:100600009300F0003B8720001302120093022000A9
:10061000E31252FE9303A001631C7704930130029E
:100620009300F0003B0110009303F000631271048B
:1006300093014002930000023B81000093030002FB
:100640006318710293015002BB0000009303000085
:100650006390700293016002930000011301E001B6
:100660003B8020009303000063147000631030028D
:100670000F00F00F638001009391110093E11100CE
:100680009308D00513850100730000000F00F00FE0
:10069000930110009308D0051305000073000000BB
:1006A000731000C000000000000000000000000007
:0C06B0000000000000000000000000003E
:1010000000000000000000000000000000000000E0
:1010100000000000000000000000000000000000D0
:1010200000000000000000000000000000000000C0
:1010300000000000000000000000000000000000B0
:081040000000000000000000A8
:040000058000000077
:00000001FF
